:03000000022DB519
:0C2DB50078FFE4F6D8FD758154022DFC77
:100E9E000A53746172743A20004950436F6E6E6546
:100EAE0063745245510A004950436F6E6E65637408
:100EBE00003E432C562C43432CC0E4E0EFF2E5F009
:100ECE0020D1E8EDEAEEEC49500A003E432C4D41AC
:100EDE00432C25303262583A25303262583A25304A
:100EEE003262583A25303262583A25303262583AD8
:100EFE0025303262582C4D414320E0E4F0E5F10AF2
:100F0E00003E432C5645522C20332E3120EEF2203B
:100F1E0025732025732CC2E5F0F1E8FF20495020FF
:100F2E00ECEEE4F3EBFF0A004E6F76203033203206
:100F3E003030370030383A35323A3335003E432CB4
:100F4E004C442C50524F473A202020202020202065
:100F5E002020202020202020202020202020202083
:100F6E002020202020202020202020202020202073
:100F7E002020202020202020202020202020202063
:100F8E00202020202020202020202020202CC4E0E3
:100F9E00F2E020EFF0EEF8E8E2EAE828F4E0E9EB20
:100FAE00290A003E2A2C312CCEF1EDEEE2EDFBE5C6
:100FBE0020EFE0F0E0ECE5F2F0FB20F1E5F2E5E207
:100FCE00EEE3EE20E8EDF2E5F0F4E5E9F1E00A00FB
:100FDE003E412C4130312C2562752E2562752E2511
:100FEE0062752E2562752C495020E0E4F0E5F12063
:100FFE00E0E4E0EFF2E5F0E00A003E412C41303251
:10100E002C2562752E2562752E2562752E2562752C
:10101E002C495020E0E4F0E5F120EEF1ED2E20F128
:10102E00E5F0E2E5F0E00A003E412C4130332C259C
:10103E0062752E2562752E2562752E2562752C49D8
:10104E005020E0E4F0E5F120F0E5E72E20F1E5F0A8
:10105E00E2E5F0E00A003E412C4130342C25627569
:10106E002E2562752E2562752E2562752CCCE0F12B
:10107E00EAE020F1E5F2E80A003E412C4130352C41
:10108E002562752E2562752E2562752E2562752CAC
:10109E00D8EBFEE70A003E532C4130362C25627504
:1010AE002CC2F0E5ECFF20EEE6E8E42E20EAE2E8C2
:1010BE00F2E0EDF6E8E820282A3130ECF1290A00BA
:1010CE003E2A2C312CC4EEEF2E20EFE0F0E0ECE5C2
:1010DE00F2F0FB20F1E5F2E5E2EEE3EE20E8EDF2D0
:1010EE00E5F0F4E5E9F1E00A003E422C5330312CF4
:1010FE002562752CC6E4E0F2FC20E7E0EFF0EEF19D
:10110E00E020F1EEE5E4E8EDE5EDE8FF20EEF2207B
:10111E00F1E5F0E2E5F0E00A003E422C5330322CCD
:10112E002562752CCEE1ECE5ED20F120F1E5F0E243
:10113E00E5F0EEEC20E1E5E720EAE2E8F2E0EDF69C
:10114E00E8E90A003E422C5330332C2562752CCF31
:10115E00E5F0E5E7E0EFF3F1EA20EFF0E820EFEE5F
:10116E00F2E5F0E520F1E2FFE7E820F120F1E5F00D
:10117E00E2E5F0EEEC0A003E422C5330342C2562B0
:10118E00752CCDE5F220EFE5F0E5E4E0F7E820E49C
:10119E00E8E0E3EDEEF1F2E8EAE820E220F1E5F036
:1011AE00E2E5F00A003E422C5330352C2562752CB8
:1011BE00CAE0EDE0EB20F8E8F0EEEAEEE2E5F8E06A
:1011CE00F2E5EBFCEDEEE3EE20EEE1ECE5EDE00A10
:1011DE00003E532C5330362C253032625825303297
:1011EE0062582530326258253032625825303262CC
:1011FE005825303262582C4D414320E0E4F0E5F1A1
:10120E0020F8E8F0EEEAEEE2E5F8E0F2E5EBFCEDD0
:10121E00EEE3EE20EEE1ECE5EDE00A003E454E4455
:10122E000A0044756D705820202020203030203068
:10123E0031203032203033203034203035203036DB
:10124E0020303720303820303920304120304220B5
:10125E0030432030442030452030460A003A2000EA
:10126E000A0044756D70442020202020303020303C
:10127E00312030322030332030342030352030369B
:10128E002030372030382030392030412030422075
:10129E0030432030442030452030460A00457272DB
:1012AE00206B657900526420656570726F6D0A005F
:1012BE005264204D454D0A00526420436F64650A06
:1012CE000044656275674950204F4E0A00446562BE
:1012DE0075674950204F46460A004465627567554A
:1012EE00736572204F6E0A004465627567557365AB
:1012FE0072204F46460A0044656275674D7367203B
:10130E004F6E0A0044656275674D7367204F4646FF
:10131E000A00436F6E666967206C6F636B210A006B
:10132E00577220656570726F6D0A00205361766585
:10133E0020656570726F6D210A00457272204D41F5
:10134E004321004C6F61643E3E002A003C41303127
:10135E003D003C4130323D003C4130333D003C418C
:10136E0030343D003C4130353D003C4130363D008F
:10137E004E4F4950004C494E4B434F4E5452005421
:10138E0052415353004652004E4F4C494E4B00496A
:10139E004E49004E4F4449414700003C21003C530A
:1013AE0030313D003C5330323D003C5330333D0034
:1013BE003C5330343D003C5330353D003C533036C9
:1013CE003D00FF137EFF1383FF138DFF1393FF1357
:0A13DE0096FF139DFF13A1FF13A853
:0635CE00010B00010900E1
:10363900C2AFC28E438910758BFF758DB7D2ABD2DD
:043649008ED2AF224C
:03001B00022C8232
:102C8200C0E0C083C082C0D0C2AFC28E758BFF7558
:102C92008DB720060675A61E75A6E10509D202E5C6
:102CA2000B6002050BE50AD394014002150A050EDA
:102CB200E50E540F7050D20DE50E543F701AD2003B
:102CC20090668DE0601204F0E0D394B4400A9080E4
:102CD200007480F0C2AF80FE906688E0600204F06B
:102CE200906104E0600214F090668EE0D39401409B
:102CF20003E014F0300502050CE50DD394644004A2
:102D0200D2068002050DE508D3940140021508D2CF
:0C2D12008ED2AFD0D0D082D083D0E0327F
:10088100C291C290D2B5C20A7D027C007F071235A7
:10089100B18F24E524646060097D017F60123569B0
:1008A100D20AE4FDFC7F0B1235B18F24E52430E63A
:1008B100097D04E4FF12358DD20A7D017C007F079A
:1008C1001235B18F24E5247008FD7FFF123569D2FE
:1008D1000A300A03126000C2AFC288C2A8C2AA7558
:1008E10089001230D5906341E0B4FA09A3E064CEE7
:1008F1007003020981E4F52474392524F582E43476
:1009010063F583E4F00524E524B443EC906341747A
:10091100FAF0A374CEF0A374CCF0906347740AF09C
:10092100E4A3F0A304F0A3F090634C7403F0A37468
:10093100CCF090633D74FFF0A3F0A3F0E4A3F0903A
:1009410063587405F0E4F524E5242401FFE433FE43
:1009510074392524F582E43463F583E0FD123620F1
:100961000524E524C3944340DFE4F5A775A61E756D
:10097100A6E1907FF0F0A3F09080007480F080FEFB
:10098100D2AF90634C7403F0A374CCF0E490634B4A
:10099100F01226F6EF6003121CDCC2B5123433C22A
:1009A10006123382906358E0C3940350037403F03A
:1009B100D20AC20CC20BD293200A077E0E7F9E126E
:1009C10027DCE4906578F0123639C2AFA37408F0E1
:1009D1009062B77424F0E4A3F0906341E09062B9AF
:1009E100F0906342E09062BAF0906343E09062BBA2
:1009F100F0906344E09062BCF0906345E09062BD8A
:100A0100F0906346E09062BEF0750A01E490657A69
:100A1100F0C207C208D2AF75A70775A61E75A6E179
:100A2100200A18AF24FE7D031228BDE4FF122BD843
:100A31007E637F78E4FB7D0112299790668DE060EB
:100A4100037401F0E4906104F0A37455F0A3748180
:100A5100F0E4F50CE4F50D906104E0700312353D0E
:100A610090668EE0B401119080007410F0E49066FD
:100A71008EF0D20AD20BD20C908008E0F52430E43B
:100A810005D2077410F0E52430E508D209908008FA
:100A91007420F0E52430E608D2089080087440F014
:100AA100E50CD394034023908002E4F0908001F0A0
:100AB100908000F0E50CD39406400FE4F50CC203DE
:100AC10090657AF0750A011233829080A0E070037C
:100AD1001231CE9080B8E070031232489080D0E09D
:100AE10070031232C2908000E0701330071012259B
:100AF10000906334EFF0D3940040031200269080FD
:100B010002E07006908000E06005D205020A55C23D
:100B110005E4F50C906104E06003020A5530091206
:100B210012239A906334EFF0D394004005E0FF1252
:100B3100001F200803020CB4122225906334EFF049
:100B41007003020A55906378E054BF247F7003025A
:100B51000C17147003020BEF24026003020C4A20ED
:100B61000A077E0E7FA71227DC300E7920037690CC
:100B71006350E07006906354E0605B906684E0FF30
:100B8100906350E0B50724906685E0FE906351E0E4
:100B9100B50618906686E0FE906352E0B5060C90AB
:100BA1006687E0FE906353E06E602B906354E06FC4
:100BB1007033906685E0FF906355E0B50727906636
:100BC10086E0FF906356E0B5071B906687E0FF90D3
:100BD1006357E0B5070F90657A7401F01200207534
:100BE1000A01020CB490668474FFF0020CB49066A2
:100BF1008DE060037401F090667CE0FF90637AE021
:100C01006F6003020CB490667CE004F0E4F50A9096
:100C11006578F0020CB4300303020CB4906347E032
:100C21007003020A55123660D203E4F50A90657822
:100C3100F090668804F0E490667BF0A3F0200A73DC
:100C41007E0E7FB51227DC806A90668DE0600374AA
:100C510001F0300352906378E020E74B90637AE033
:100C6100FF90667BE0FE6F600D906683E07007EE9B
:100C7100146F703F801390667BE004F0906334E062
:100C8100FFD394044003122A6B9060007482F0A396
:100C91007401F090637AE0906002F07E607F007DE5
:100CA10003123153020A55300E092003069066845F
:100CB10074FFF0200303020D69E50A706B122D1E0B
:100CC100EF60207E647F78906479E02404FD123126
:100CD10053906683E06003020A55906358E0F50A79
:100CE100020A55906688E0D3943C403C906683E0CC
:100CF100703690668804F09062B6E0702B122B2358
:100D0100E4906478F0A37412F090667CE090647AC9
:100D1100F0A374FDF090610763A20190647C63A26B
:100D2100017F12121FAA809B12364DEF6015906051
:100D3100007483F0E4A3F07E607F007D02123153E2
:100D4100020A55E50A64016003020A55906578E0DC
:100D510004F0E0C394055003020CC4C203E490659F
:100D61007AF0120020020A55E50A64016003020AC2
:100D71005590657AE014604024FE603C14700302D3
:100D81000E5124046003020A55E4F50C200E139061
:100D9100657A7404F0906578E05401F0750A0102F7
:100DA1000A55E490657AF090657804F0750AC89068
:100DB100668474FFF0020A55906684E07003020EA7
:100DC100409064787480F090647A7401F0E4A3F048
:100DD100A304F0A37430F0A3747BF0E4F524747FD2
:100DE1002524F582E43464F583747DF07480252430
:100DF100F582E43464F583E4F0E524240790647912
:100E0100F07C667D8490634CE0FAA3E0FB7F0212E4
:100E11002F517E647F78E5242409FD1231539066B9
:100E210083E0601B123660D203E4F50A906578F026
:100E310090668804F0E490667BF0A3F0020A559076
:100E4100657A7404F0906358E02432F50A020A5579
:100E51009080027410F0750A03906578E06401FFD8
:100E6100F090657A7401F0EF7019906354E06013AB
:100E7100FCA3E0FDA3E0FEA3E0FF906684121B9EAD
:100E8100020A55906350E0FCA3E0FDA3E0FEA3E05D
:0C0E9100FF906684121B9E020A5580FE32
:010E9D002232
:10002600906379E0B444047F0180027F0090637896
:10003600E0B447047E0180027E00EE5F604A906372
:1000460041E090637AF0906342E090637BF09063C6
:1000560043E090637CF0906344E090637DF09063AE
:1000660045E090637EF0906346E090637FF0906396
:10007600797452F09062B063A2019080A863A201E5
:100086007F06121FAA020877906334E0C3940850D3
:1000960003020880906341E0FF90637AE06F60039B
:1000A600020880906342E0FF90637BE06F6003028A
:1000B6000880906343E0FF90637CE06F6003020872
:1000C60080906344E0FF90637DE06F6003020880E8
:1000D600906345E0FF90637EE06F600302088090C6
:1000E6006346E0FF90637FE06F60030208809063E1
:1000F60079E0B444159062B0E0B4FF0E63A20190BB
:1001060080A863A2017F06121FAA90668DE0600395
:100116007401F090668E7464F09063797452F09076
:100126006378E0646D60030202A37BFF7A0E79BFF9
:1001360012144A7BFF7A0E79D9906341E0F52DA31C
:10014600E0F52EA3E0F52FA3E0F530A3E0F531A30B
:10015600E0F53212144A752DFF752E0F752F367580
:1001660030FF75310F7532427BFF7A0F790F12140B
:100176004A7BFF7A0F794B12144A7BFF7A0F79B1CB
:1001860012144A7BFF7A0F79DE906347E0F52DA3C0
:10019600E0F52EA3E0F52FA3E0F53012144A7BFF1D
:1001A6007A107908906350E0F52DA3E0F52EA3E0D0
:1001B600F52FA3E0F53012144A7BFF7A10793690BA
:1001C6006354E0F52DA3E0F52EA3E0F52FA3E0F5AB
:1001D6003012144A7BFF7A10796490633DE0F52D66
:1001E600A3E0F52EA3E0F52FA3E0F53012144A7B29
:1001F600FF7A107987906339E0F52DA3E0F52EA3F9
:10020600E0F52FA3E0F53012144A7BFF7A1079A4AB
:10021600906358E0F52D12144A7BFF7A1079CE12BE
:10022600144A7BFF7A1079F7A20EE433F52D1214E7
:100236004A7BFF7A117927906683E0F52D12144ADE
:100246007BFF7A11795290668DE0F52D12144A7B68
:10025600FF7A1179859062B6E0F52D12144A7BFF7C
:100266007A1179B3A201E433F52D12144A7BFF7A91
:100276001179DF90667DE0F52DA3E0F52EA3E0F57C
:100286002FA3E0F530A3E0F531A3E0F53212144ACE
:100296001233DB7BFF7A12792A12144A2290637892
:1002A600E0644C70527E127F301227DC906380E04F
:1002B600F525A3E0F526E4F5277D03AF26AE251246
:1002C60028BD7E127F6B1227DCAE25AF26E4FB7DB0
:1002D600101229977E127F6E1227DC74102526F5E0
:1002E60026E43525F5250527E527C3941040CA7E63
:1002F600127F6E1227DC22906378E0646C705CF5E6
:10030600297E127F701227DCE4F528AF297E007D56
:10031600031228BD7E127F6B1227DCE4F527A8297D
:10032600E6FF74822527F582E43463F583EFF00552
:10033600290527E527B410E67E637F82E4FB7D105E
:100346001229977E127F6E1227DC0528E528C394B2
:100356000840B87E127F6E1227DC22906378E06434
:100366004B7061F527746A2527F582E43463F583BB
:10037600E06032746A2527F582E43463F583E0F49D
:100386006023746A2527F582E43463F583E0FF74FD
:10039600802527F582E43463F583E0B50710052749
:1003A600E527B408C09061047432F00208779063C0
:1003B600787421F0300A030208777E127FAB122789
:1003C600DC020877906378E0B4521A200A077E129E
:1003D6007FB31227DC9063787472F07E637F787D3A
:1003E60008122FD522906378E064497045200A07E9
:1003F6007E127FBE1227DC906380E0F525A3E0F530
:1004060026E4F527852682852583E0FF7482252745
:10041600F582E43463F583EFF00526E526700205E0
:10042600250527E527B480DC7E637F787D8A122F39
:10043600D522906378E064437079A3E064527046F5
:10044600200A077E127FC61227DC906380E0F5251E
:10045600A3E0F526E4F527852682852583E493FF28
:1004660074822527F582E43463F583EFF00526E5EB
:1004760026700205250527E527B480DB7E637F7895
:100486007D8A122FD522906379E0645760030208B3
:1004960080906380E0F525A3E0F52674822527F594
:1004A60082E43463AD82FC7B80AF26AE251235092B
:1004B600020877906378E06444600302054A90631B
:1004C60080E0FF64447003020877EFB4310CC20A7F
:1004D6007E127FCF1227DC020877906380E0B4306B
:1004E6000CD20A7E127FDB1227DC0208779063802B
:1004F600E0B4320CD20B7E127FE81227DC020877BA
:10050600906380E0B4330CC20B7E127FF61227DCB8
:10051600020877906380E0B4340CD20C7E137F051A
:100526001227DC020877906380E0B4350CC20C7E9B
:10053600137F121227DC020877906380E0FF120017
:100546001E020877906104E07013200A077E137F6D
:10055600201227DC9063787421F0020877906104FA
:100566007432F0906378E0FFB4510A908000748092
:10057600F0C2AF80FEEF64577045200A077E137FF6
:100586002E1227DC906381E0906334F0E4F5279027
:100596006334E0FFE527C39F400302087774822592
:1005A60027F582E43463F583E0FF906380E0252736
:1005B60024AFF582E43461F583EFF0052780D0900F
:1005C6006378E064536003020679200A077E137F8E
:1005D600391227DC906341E0FF9061B8E06F703C10
:1005E600906342E0FF9061B9E06F7030906343E042
:1005F600FF9061BAE0B50724906344E0FF9061BBC9
:10060600E0B50718906345E0FF9061BCE0B5070CC4
:10061600906346E0FF9061BDE06F6016906378746A
:1006260021F0300A030208777E137F481227DC0286
:100636000877E4F527E4F50DAF27FE74AF2527F517
:1006460082E43461F583E0FD1236200527E527C3F1
:1006560094FE40E19080007480F0C2AFE4907FF099
:10066600F0A3F0907FFD74AAF0A374FFF0A3745575
:10067600F080FE906378E0644F704C906380E0F504
:1006860025A3E0F526E5264525700A200A077E13F0
:100696007F511227DC200A077E137F581227DCE4DD
:1006A600F52774822527F582E43463F583E08526F1
:1006B60082852583F00526E526700205250527E5B2
:1006C60027B480DE020877906378E0FFB445279070
:1006D60080007480F0906380E0FDA3E0907FF0CD11
:1006E600F0A3EDF0C2AF907FFD74AAF0A374FFF003
:1006F600A37455F080FEEF6465600302087790638B
:1007060080E0FFA3E0907FF0CFF0A3EFF0E4F525C3
:10071600F526D3907FF1E09526907FF0E095254071
:1007260020E4F50D2526FFE5253401FE8526828584
:100736002583E0FD1236200526E526700205258074
:10074600D17E137F5A122ECCEF4E602012000390FA
:100756006347EFF0120003906348EFF01200039036
:100766006349EFF012000390634AEFF07E137F6057
:10077600122ECCEF4E6020120003906350EFF01261
:100786000003906351EFF0120003906352EFF012F2
:100796000003906353EFF07E137F66122ECCEF4E6C
:1007A6006020120003906354EFF01200039063552B
:1007B600EFF0120003906356EFF0120003906357B8
:1007C600EFF07E137F6C122ECCEF4E6020120003EA
:1007D60090633DEFF012000390633EEFF0120003CA
:1007E60090633FEFF0120003906340EFF07E137FBB
:1007F60072122ECCEF4E6020120003906339EFF098
:1008060012000390633AEFF012000390633BEFF09F
:1008160012000390633CEFF07E137F78122ECCEF2C
:100826004E6008123325906358EFF0E4F527E4F59F
:100836000DE5272401FFE433FE74392527F582E40C
:100846003463F583E0FD1236200527E527C394437C
:1008560040DC9080007480F0C2AFE4907FF0F0A39B
:10086600F0907FFD74AAF0A374FFF0A37455F08096
:0A087600FE7E637F787D08122FD507
:010880002255
:1034D100AE07EEC39430400BEED394395005EE2481
:1034E100D0FF22EEC39461400BEED394665005EEFB
:1034F10024A9FF22EEC39441400BEED3944650051C
:08350100EE24C9FF22AF0622EF
:103606009062AFE004F070069062AEE004F0906263
:0A361600AEE0FEA3E0FF1235EA2249
:100003001236061234D1EFC454F0FEC0061236067F
:080013001234D1D0E02FFF22CE
:10332500E49068B2F01236069068B3EFF0C39430BB
:103335004018E0FFD3943950119068B2E02407F5A6
:1033450082E43461F583EFF080119068B2E02407E0
:10335500F582E43461F583E4F0800C9068B2E00412
:10336500F0E0D3940840BE752D00752E00752F0032
:0C337500E4F5307B017A617907122081B9
:013381002229
:042ECC008E2A8F2B90
:102ED0009062AEE4F0A374FFF0123606EF606EF479
:102EE000606B852B82852A83E493B507EC752C01F2
:102EF000E52B252CF582E4352AF583E493602590B3
:102F000062AFE0252CFF9062AEE03400FE1235EA9D
:102F1000E52B252CF582E4352AF583E493B50704E7
:102F2000052C80CCE52B252CF582E4352AF583E4AD
:102F30009370A6E52C24FFFFE434FFFE9062AFE01F
:102F40002FF09062AEE03EF07E007F0122E4FEFFB3
:012F5000225E
:1026F6007E137FA9122ECCEF4E70037F01227E132C
:102706007FAC122ECCEF4E600C123606EF24D0248E
:10271600FF920E8002D20E7E137FB2122ECCEF4EA7
:10272600600C123606EF24D0906683F08005E490A4
:102736006683F07E137FB8122ECCEF4E600C1236F5
:1027460006EF24D090668DF08005E490668DF07ECD
:10275600137FBE122ECCEF4E600C123606EF24D03D
:102766009062B6F08005E49062B6F07E137FC412E4
:102776002ECCEF4E600C123606EF24D024FF9201C9
:102786008002C20190634163A20190667D63A2014B
:102796007F06121FAA30013B7E137FCA122ECCEF92
:1027A6004E603012000390667DEFF01200039066D3
:1027B6007EEFF012000390667FEFF0120003906642
:1027C60080EFF0120003906681EFF012000390662E
:0627D60082EFF07F0022FB
:101CDC00C201E490668DF0D20EC204906683F0903F
:101CEC0062B6F090634163A20190667D63A2017FAE
:101CFC0006121FAAE4F525E52575F003A424D0F5FA
:101D0C0082E43413F583E493FB740193FA74029325
:101D1C00F9121A6B7003021ECEE4F526F527FD743A
:101D2C002F2DF582E43461F583E0FF7003021EC9A8
:101D3C00E52575F003A424D0F582E43413F583E48F
:101D4C0093FB740193FA740293F9852682758300D0
:101D5C00121A84FEEFB506087527010526021EC56A
:101D6C00E5277003021EC5EE6003021EC0E52524A4
:101D7C00FE6028147003021EA8147003021EAC141B
:101D8C007003021EB4147003021EB8240560030213
:101D9C001EC990668D7401F0021EC9D201742F2DDC
:101DAC00F582E43461F583E0FF642D7003021EC9F3
:101DBC001234D1EFC454F0FC74302DF582E434614C
:101DCC00F583E0FF1234D1EF2C90667DF074312D49
:101DDC00F582E43461F583E0FF1234D1EFC454F0A2
:101DEC00FC74322DF582E43461F583E0FF1234D1BA
:101DFC00EF2C90667EF074332DF582E43461F5831C
:101E0C00E0FF1234D1EFC454F0FC74342DF582E4AD
:101E1C003461F583E0FF1234D1EF2C90667FF074BF
:101E2C00352DF582E43461F583E0FF1234D1EFC433
:101E3C0054F0FC74362DF582E43461F583E0FF1226
:101E4C0034D1EF2C906680F074372DF582E4346138
:101E5C00F583E0FF1234D1EFC454F0FC74382DF547
:101E6C0082E43461F583E0FF1234D1EF2C9066816B
:101E7C00F074392DF582E43461F583E0FF1234D12E
:101E8C00EFC454F0FC743A2DF582E43461F583E030
:101E9C00FF1234D1EF2C906682F08021D204801D89
:101EAC009066837401F08015C20E80119062B67436
:101EBC0001F08009E4F527F5260D021D2B052502FE
:021ECC001D03F4
:011ECE0022F1
:10348A00906579E0C3947C503D906579E0FE04F044
:10349A0074B72EF582E43462F583EFF0BF0A279001
:1034AA006579E0FF04F074B72FF582E43462F5839E
:1034BA00E4F0906579E0FF1230579065797408F06E
:0734CA009062B8E004F0225B
:103382009080007480F090633963A201F583F58226
:1033920063A2017F08121FAA90634163A201908079
:1033A2008863A2017F0A121FAA908092E4F0A3749C
:1033B20032F0A37401F090634BE0FF9080B1F09083
:1033C20080E1EFF09080957455F0A3F09080007446
:0933D20001F09080097470F022F2
:1031CE00908009E04410F09080A0E0706C9080A197
:1031DE007482F09080A874FFF0A3F0A3F0A3F07FA8
:1031EE00039080AEEFF07FCBA3EFF07F039080AC27
:1031FE00EFF0A374CBF09080007402F09068A612EA
:10320E001BAA000000009068A6E0908040F0906835
:10321E00A7E0908041F09068A8E0908042F090681E
:10322E00A9E0908043F0A3E4F0A3F0A3F0A3F09004
:09323E008018F0A3F0A3F0A3F046
:013247002264
:1032C200908009E04440F09080D17482F090634C89
:1032D200E0FF9080DEF090634DE0FF9080DFF090A1
:1032E20080027402F09068AA121BAA0000000090EB
:1032F20068AAE0908058F09068ABE0908059F09016
:1033020068ACE090805AF09068ADE090805BF0A3EA
:10331200E4F0A3F0A3F0A3F0908030F0A3F0A3F0C8
:02332200A3F016
:013324002286
:10324800908009E04420F09080B8E0706C9080B9DC
:103258007482F07F039080C6EFF07FCDA3EFF07FFC
:10326800039080C4EFF0A374CDF09080C074FFF099
:10327800A3F0A3F0A3F09080017402F09068AE125E
:103288001BAA000000009068AAE090804CF09068AB
:10329800ABE090804DF09068ACE090804EF0906884
:1032A800ADE090804FF0A3E4F0A3F0A3F0A3F0907A
:0932B8008024F0A3F0A3F0A3F0C0
:0132C10022EA
:102F51008C258D26A907EAFDE975F018A424ACFF9C
:102F6100E5F034808F82F583EDF0EBFDE975F01823
:102F7100A4FFAEF024ACFBEE34808B82F583A3ED8D
:102F8100F08526828C83E0FDEF24A8FFEE3480FEDD
:102F91008F82F583EDF08526828C83A3E08F828E6C
:102FA10083A3F0852682852583A3A3E0FDE975F03F
:102FB10018A424A8FFE5F03480FE8F82F583A3A333
:102FC100EDF08526828C83A3A3A3E08F828E83A359
:042FD100A3A3F022A4
:062FD5008D2AAB07AA06DD
:102FDB009068A6E0FCA3E0FDA3E0FEA3E0F52E8E37
:102FEB002D8D2C8C2BAE02AF038E838F8263A201AF
:102FFB00E52D540744C0F583852E8263A201AF2AC9
:10300B00122013908000E020E5F9E4FCFDFEE52E94
:10301B00252AF52EEE352DF52DED352CF52CEC3531
:10302B002BF52B908040E52BF0A3E52CF0A3E52DA1
:10303B00F0A3E52EF09080007420F0AF2EAE2DADF6
:0B304B002CAC2B9068A6121B9EAF2A35
:013056002257
:063153008D25AB07AA0662
:103159009068AAE0FCA3E0FDA3E0FEA3E0F5298EB8
:10316900288D278C26AE02AF038E838F8263A2013E
:10317900E528540744D0F58385298263A201AF2548
:10318900122013E4FCFDFEE5292525F529EE352855
:10319900F528ED3527F527EC3526F526908058E5F5
:1031A90026F0A3E527F0A3E528F0A3E529F0908010
:1031B900027420F0AF29AE28AD27AC269068AA1278
:0431C9001B9EAF2575
:0131CD0022DF
:022BD8008F2547
:102BDA00908001E030E5037F00229068AEE0FCA31C
:102BEA00E0FDA3E0FEA3E0F5298E288D278C269030
:102BFA00667D63A201E528540744C8F583852982C6
:102C0A0063A2017F06122029E5292406F529E43565
:102C1A0028F528E43527F527E43526F52690657B3F
:102C2A0063A201E528540744C8F58385298263A273
:102C3A0001AF25122029E4FCFDFEE5292525F52909
:102C4A00EE3528F528ED3527F527EC3526F52690BB
:102C5A00804CE526F0A3E527F0A3E528F0A3E529B3
:102C6A00F09080017420F0AF29AE28AD27AC2690F1
:072C7A0068AE121B9EAF259E
:012C81002230
:102500009081E0E0F525052505250525052505250E
:1025100005250525052505250525908010E0F528CC
:10252000A3E0F529A3E0F52AA3E0F52B9081E1E0F3
:10253000F52505250525052505250525052505255B
:10254000052505250525908014E0F52CA3E0F52D43
:10255000A3E0F52EA3E0F52FE52EB52A08E52FB56B
:102560002B037F0022E4F525E52E540744E0F58394
:10257000852F8263A20190637863A2017F081220F5
:102580004190637A63A2019062B063A2017F061258
:102590001FAA906378E0F526A3E0F527E4F52590DF
:1025A0006378E0702AA3E024F8F525E52E5407446B
:1025B000E0F583852F8274082582F582E43583F562
:1025C0008363A20190637863A201AF25122041AE1C
:1025D00026E4FCFDE52F2527F52FE52E3EF52EED13
:1025E000352DF52DEC352CF52C908014E52CF0A331
:1025F000E52DF0A3E52EF0A3E52FF09080007440C8
:03260000F0AF2513
:0126030022B4
:102225009081E6E0F52505250525052505250525E6
:1022350005250525052505250525908028E0F52892
:10224500A3E0F529A3E0F52AA3E0F52B9081E7E0CB
:10225500F525052505250525052505250525052539
:1022650005250525052590802CE0F52CA3E0F52D09
:10227500A3E0F52EA3E0F52FE4F525E52EB52A0A12
:10228500E52FB52B05C20802237FE52E540744F040
:10229500F583852F8263A20190637863A2017F088D
:1022A500122041906378E0F526A3E0F527E5274560
:1022B5002670099080027410F07F0022906684E0F9
:1022C500FFF4602D90637AE06F7076906685E0FF8D
:1022D50090637BE06F706A906686E0FF90637CE0B8
:1022E5006F705E906687E0FF90637DE06F6022808F
:1022F5005090637AE0906684F090637BE090668509
:10230500F090637CE0906686F090637DE090668750
:10231500F0906378E0702AA3E024F8F525E52E54C3
:102325000744F0F583852F8274082582F582E4350C
:1023350083F58363A20190637863A201AF25122020
:1023450041AE26E4FCFDE52F2527F52FE52E3EF5CC
:102355002EED352DF52DEC352CF52CAF2BAE2AAD0C
:1023650029AC28AB2FAA2EA92DA82CD3121B8D4042
:10237500099080027410F07F002290802CE52CF0EB
:10238500A3E52DF0A3E52EF0A3E52FF090800274D0
:0423950040F0AF2540
:012399002221
:10239A009081E3E0F5250525052505250525052573
:1023AA000525052505250525052590801CE0F52828
:1023BA00A3E0F529A3E0F52AA3E0F52B9081E4E058
:1023CA00F5250525052505250525052505250525C3
:1023DA00052505250525908020E0F52CA3E0F52D9F
:1023EA00A3E0F52EA3E0F52FE4F525E52EB52A0A9C
:1023FA00E52FB52B05C2090224E5E52E540744E86A
:10240A00F583852F8263A20190600463A2017F0E87
:10241A00122057906004E0F526A3E0F52790600C9F
:10242A00E0FFF4604590667DE0FEEF6E706EA3E01B
:10243A00FF90600DE06F706490667FE0FF90600E21
:10244A00E06F7058906680E0FF90600FE06F704C0C
:10245A00906681E0FF906010E06F7040906682E0C5
:10246A00FF906011E06F60048032D2D9906004E07E
:10247A00702AA3E024F2F525E52E540744E8F583F3
:10248A00852F82740E2582F582E43583F58363A253
:10249A000190600463A201AF25122057AE26E4FC26
:1024AA00FDE52F2527F52FE52E3EF52EED352DF5E9
:1024BA002DEC352CF52CAF2BAE2AAD29AC28AB2F41
:1024CA00AA2EA92DA82CD3121B8D5006E527452626
:1024DA0070099080017410F07F0022908020E52C12
:1024EA00F0A3E52DF0A3E52EF0A3E52FF0908001EF
:0524FA007440F0AF2565
:0124FF0022BA
:0427DC008E2A8F2B87
:1027E0009068A6E0FCA3E0FDA3E0FEA3E0F5318E37
:1027F000308D2F8C2EE531FFE5305407FEE42FF5A8
:102800002DEE34C0F52C852D82F5837423F0052D33
:10281000E52D7002052C532CC7F582852C83740A94
:10282000F0052DE52D7002052C532CC790634163F4
:10283000A201852C83852D8263A2017F06122013BD
:102840007406252DF52DE4352CF52C852A83852B52
:102850008263A201852C83852D8263A201121FF75A
:10286000908000E020E5F9E4FCFDFE9068A6E0F829
:10287000A3E0F9A3E0FAA3E02FFFEE3AFEED39FD65
:10288000EC38FCEF2408FFE43EFEE43DFDE43CFCB4
:102890009068A6121B9E9068A6E0908040F0906819
:1028A000A7E0908041F09068A8E0908042F09068A6
:0C28B000A9E0908043F09080007420F0BC
:0128BC0022F9
:062997008E2A8F2B8D2C0F
:10299D009068A6E0FCA3E0FDA3E0FEA3E0F5328E77
:1029AD00318D308C2FE532FFE5315407FEE42FF5E4
:1029BD002EEE34C0F52D852E82F5837423F0052E71
:1029CD00E52E7002052D532DC7F582852D83EBF075
:1029DD00052EE52E7002052D532DC790634163A280
:1029ED0001852D83852E8263A2017F06122013742B
:1029FD0006252EF52EE4352DF52D852A83852B8282
:102A0D0063A201852D83852E8263A201AF2C122036
:102A1D0013908000E020E5F97408252CF52CFFE4D7
:102A2D00FCFDFEE5322FF532EE3531F531ED353069
:102A3D00F530EC352FF52F908040E52FF0A3E530E4
:102A4D00F0A3E531F0A3E532F09080007420F0AFF3
:0D2A5D0032AE31AD30AC2F9068A6121B9E3A
:012A6A002249
:023057008F3EAA
:103059009068A6E0FCA3E0FDA3E0FEA3E0F5428EA4
:10306900418D408C3FE542FFE5415407FEE42FFFC7
:10307900EE34C09062B763A201F5838F8263A20127
:10308900AF3E122013908000E020E5F9E4FCFDFE3C
:10309900E542253EF542EE3541F541ED3540F54035
:1030A900EC353FF53F908040E53FF0A3E540F0A3C4
:1030B900E541F0A3E542F09080007420F0AF42AE04
:0B30C90041AD40AC3F9068A6121B9E7A
:0130D40022D9
:0628BD008E2A8F2BAB05F3
:1028C3009068A6E0FCA3E0FDA3E0FEA3E0F5318E53
:1028D300308D2F8C2EE531FFE5305407FEE42FF5C4
:1028E3002DEE34C0F52C852D82F5837423F0052D50
:1028F300E52D7002052C532CC7F582852C83EBF054
:10290300052DE52D7002052C90634163A201852CF2
:1029130083852D8263A2017F061220137406252D61
:10292300F52DE4352CF52C532CC7E52A852D82850E
:102933002C83F0052DE52D7002052C532CC7F58251
:10294300852C83E52BF0052DE52D7002052C532CEA
:10295300C7908000E020E5F9E531240AF531E4353C
:1029630030F530E4352FF52FE4352EF52E908040E9
:10297300E52EF0A3E52FF0A3E530F0A3E531F090C9
:1029830080007420F0AF31AE30AD2FAC2E9068A62E
:03299300121B9E76
:01299600221E
:1035EA00E5D220E0FBC2AF438E2075D2028F828ED5
:0B35FA0083E0FFE4F5D2538EDFD2AF78
:0136050022A2
:10362000E5D220E0FBC2AF43D2028F828E83EDF061
:0936300075D25063D250D2AF22D2
:1030D500E4FDED2401FFE433FE1235EA74392DF5E4
:1030E50082E43463F583EFF00DBD3FE6E4FDED24A6
:1030F5007FFFE433FE1235EA742F2DF582E4346147
:10310500F583EFF0742F2DF582E43461F583E070DB
:103115001B742F2DF582E43461F5837420F074302F
:103125002DF582E43461F583E4F080040DBD80BEA5
:10313500E49061AEF0FDEDFF7E001235EA74AF2D2F
:0D314500F582E43461F583EFF00DBDFEE985
:01315200225A
:023509008B2A0B
:10350B00A2AF920FC2AF85A22B53A2FE8E838F82E6
:10351B0005A28C838D82740912206FE52A53A2FEBB
:10352B0043A22012207153A2DF852BA2A20F92AFD0
:01353B00FF90
:01353C00226C
:1035B100A2AF920FC2AF8C838D82EF12206F43A214
:0C35C1002012207153A2DFA20F92AFFF76
:0135CD0022DB
:023569008F25AC
:10356B00A2AF920FC2AFE4F5838D82740612206F67
:10357B00E52543A22012207153A2DFA20F92AF7F49
:01358B00013E
:01358C00221C
:02358D008F2588
:10358F00A2AF920FC2AFE4F5838D82740A12206F3F
:10359F00E52543A22012207153A2DFA20F92AF7F25
:0135AF00011A
:0135B00022F8
:101ECF00A907E7FFA805EF93C3966008403B74FC92
:101EDF002FFF80F00F08EF93C3966008402B74FB21
:101EEF002FFF80E00F08EF93C3966008401B74FA32
:101EFF002FFF80D00F08EF93D3966008400B74F933
:101F0F002FFF80C01F1F1F1F1FEF54FEF80303F783
:101F1F00E893FC08E893FD08E893FE08E893FF2296
:101F2F0009E993C39D6008402974FB29F980F109E1
:101F3F00E993C39E6008401A74FA29F980E209E90F
:101F4F0093D39F6008400B74F929F980D31919199D
:101F5F001919E9C313C313FF22740093F8ECC39844
:101F6F004024701F740193F8EDC3984019701474D6
:0E1F7F000293F8EEC398400E7009740393F8B5
:101F8D00EFC39840037F00227F0122EDF8E6F008B1
:101F9D00A3DFFA22EDF8E0F608A3DFFA22E0A3634F
:101FAD00A201F0A363A201DFF475A20022E0A363F6
:101FBD00A201F0A363A201E0A363A201F0A363A2B7
:101FCD0001E463A201F0A363A201DFE175A2002287
:101FDD00E0A363A2016DFE936CFDEE058393FC15EA
:101FED008363A201DFEA75A200227F00E493A3635D
:101FFD00A201F00F600CA3E583C2E3F58363A20198
:10200D0080EA75A20022E0A363A201F0A3E583C2DA
:10201D00E3F58363A201DFEE75A20022E0A363A2C4
:10202D0001F0A3E583C2E4D2E3F58363A201DFEC03
:10203D0075A20022E583C2E3F583E0A363A201F05C
:10204D00A363A201DFEE75A20022E583C2E4D2E311
:10205D00F583E0A363A201F0A363A201DFEC75A2F7
:10206D000022F922C002C004C00612FFF0D006D033
:04207D0004D0022267
:101744003E2A2C312CCFE0F0E0ECE5F2F0FB20E077
:10175400F1E8EDF5F0EEEDEDEEE3EE20EFEEF0F274
:10176400E00A003E4C2C4930312C256C752CD1EA12
:10177400EEF0EEF1F2FC20EEE1ECE5EDE02C35309C
:101784002C3130302C3330302C3630302C31323058
:10179400302C323430302C343830302C3936303030
:1017A4002C31393230302C33383430302C35373614
:1017B40030302C3131353230300A003E422C493041
:1017C400322C2562752CC2FBF1F2E0E2EBFFF2FC55
:1017D4002052545320EFF0E820EFE5F0E5E4E0F781
:1017E400E50A003E532C4930332C2562752CC7E0A2
:1017F400E4E5F0E6EAE020F1F2E0F0F2E020EFE5E3
:10180400F0E5E4E0F7E8282A3130ECF1290A003C5D
:1018140021003C4930313D003C4930323D003C49D7
:1018240030333D003C4930343D003C4930353D00C7
:101834003C4930363D003C4930373D003C49303866
:101844003D000AC1F3F4E5F020E7E0EDFFF22100EA
:101854000A4F55543E000A3C0020212121435243A3
:10186400204552523A20000089129B24AD36BF48CD
:10187400C15AD36CE57EF78108931AA52CB73EC9EB
:1018840040DB52ED64FF76028B109926AF34BD4ADB
:10189400C358D16EE77CF5830A9118A72EB53CCBCB
:1018A40042D950EF66FD74048D169F20A932BB4CBB
:1018B400C55ED768E17AF3850C971EA128B33ACDAB
:1018C40044DF56E960FB72068F149D22AB30B94E9B
:1018D400C75CD56AE378F1870E951CA32AB138CF8B
:1018E40046DD54EB62F97008811A932CA53EB7408B
:1018F400C952DB64ED76FF89009B12AD24BF36C16B
:1019040048D35AE56CF77E0A8318912EA73CB5425A
:10191400CB50D966EF74FD8B029910AF26BD34C34A
:101924004AD158E76EF57C0C851E9728A13AB3443A
:10193400CD56DF60E972FB8D049F16A920BB32C52A
:101944004CD75EE168F37A0E871C952AA338B1461A
:10195400CF54DD62EB70F98F069D14AB22B930C70A
:101964004ED55CE36AF17800112332465765748CD6
:101974009DAFBECADBE9F810013322564775649C5B
:101984008DBFAEDACBF9E82130021367764455AD4A
:10199400BC8E9FEBFAC8D93120120377665445BD3B
:1019A400AC9E8FFBEAD8C94253617004152736CE2A
:1019B400DFEDFC8899ABBA5243716014053726DE1B
:1019C400CFFDEC9889BBAA6372405125340617EF0A
:1019D400FECCDDA9B88A9B7362504135241607FFFB
:1019E400EEDCCDB9A89A8B8495A7B6C2D3E1F008F2
:1019F400192B3A4E5F6D7C9485B7A6D2C3F1E018DB
:101A0400093B2A5E4F7D6CA5B48697E3F2C0D129C9
:101A1400380A1B6F7E4C5DB5A49687F3E2D0C139BA
:101A2400281A0B7F6E5C4DC6D7E5F48091A3B24AA9
:101A34005B69780C1D2F3ED6C7F5E49081B3A25A9A
:101A44004B79681C0D3F2EE7F6C4D5A1B082936B89
:101A54007A48592D3C0E1FF7E6D4C5B1A092837B7A
:071A64006A58493D2C1E0FDA
:1035D40052668F00000000000000000000000000A0
:0535E4000000000000E2
:01001E0022BF
:03002300022E4169
:0B2E4100C0E0C083C082C0D075D01874
:102E4C0030984BC298750B01AF99E543700EEF6447
:102E5C0055703BF54A754301D2918032E553702E83
:102E6C0074A1254AF582E43466F583EFF0E54AB4A3
:102E7C000104EF04F544E54A600AB5440F04F55328
:102E8C00C2918008EF64556003754300054A309980
:102E9C0026301921D290E551B5490AC219D21BC26C
:102EAC0090D296801074A12551F582E43467F58395
:072EBC00E0F5990551C299F0
:092EC300D0D0D082D083D0E032DF
:1033DB007BFF7A17794412144A9068A4E0FEA3E0AD
:1033EB00FFC3E49FFFE49EFEAB07FA3395E0F9F8C9
:1033FB007F007E8C7D0A7C00121AED8F308E2F8D14
:10340B002E8C2D7BFF7A17796712144A7BFF7A1764
:10341B0079BFA21AE433F52D12144A7BFF7A177980
:08342B00E785462D12144A2228
:102604007E187F13122ECCEF4E70037F01227E18AA
:102614007F16122ECCEF4E6023123325A804A90591
:10262400AA06AB077F007E8C7D0A7C00121AED128D
:102634001B7F9068A4EEF0A3EFF0800A9068A47466
:10264400FFF0A374B8F07E187F1C122ECCEF4E60FE
:102654000C123606EF24D024FF921A8002C21A7E8E
:10266400187F22122ECCEF4E60071233258F46803E
:1026740003E4F5467E187F28122ECCEF4E60071235
:1026840033258F458003E4F5457E187F2E122ECC2A
:10269400EF4E60071233258F548003E4F5547E18FF
:1026A4007F34122ECCEF4E600A1233259068A1EFCE
:1026B400F080069068A17401F07E187F3A122ECC47
:1026C400EF4E600A1233259068A2EFF080069068FE
:1026D400A27402F07E187F40122ECCEF4E600A12D4
:1026E40033259068A3EFF080069068A37403F07F0D
:0226F4000022C2
:10343300C219C21BE4F543F551F549F54AF50BC230
:1034430018755209122604D296C2ADE4F5C9D2CD3D
:10345300D2CCC2C9C2CAF5CDF5CC9068A4E0F5CBF5
:10346300A3E0F5CA85CBCD85CACCE4F598D29E43BB
:103473008740C29FC2ACC298C29975B81075B71085
:07348300D2CAD29CD2AC2298
:01001F0022BE
:102B2300E4FF0F2407F582E43461F583E552F00FE7
:102B330074072401F582E43461F583E4F07C667D57
:102B430094FEED1DAA0470011CF5828A83E0FBAAA2
:102B5300070F74072AF582E43461F583EBF00EBEA8
:102B630004E07C667D98E4FEED1DAA0470011CF56B
:102B7300828A83E0FBAA070F74072AF582E4346193
:102B8300F583EBF00EBE04E07C667D9CE4FEED1D58
:102B9300AA0470011CF5828A83E0FBAA070F74075D
:102BA3002AF582E43461F583EBF00EBE04E07C6623
:102BB3007DA0E4FEED1DAA0470011CF5828A83E06A
:102BC300FBAA070F74072AF582E43461F583EBF05F
:042BD3000EBE04E04E
:012BD70022DB
:08365800C2992099FDD29922CC
:07366000D2CAD29CD2AC22B9
:102A6B008F2530190E300A03022B227E187F461257
:102A7B0027DC2290637BE0F5527F7C7583630582B4
:102A8B0063A2019067A463A201E52524FCFF121F3A
:102A9B00AA9067A17455F0A3F0E52524FEA3F0E5F9
:102AAB002504F549E4F54DF54EE52524FCF5507F5D
:102ABB00A4758367058263A20190186B63A201AFB3
:102ACB0050AE4FAD4EAC4D121FDD8F508E4F8D4E15
:102ADB008C4D749F2549F582E43467F583E54EF000
:102AEB0074A02549F582E43467F583E54DF0E4F5F0
:102AFB0051D219C296E5466004F508800312365888
:102B0B00200A127E187F541227DC7E677FA1E4FB1C
:082B1B00AD49122997C21B22EB
:102D1E00E5537002FF22E55324FEF5259066A3636A
:102D2E00A20190647C63A201AF25121FAAE4F543B1
:102D3E00F553906478F0E52524FEA3F090667CE0D0
:102D4E0090647AF0A37419F0E4F54DF54E85255094
:102D5E007F7C758364058263A20190186B63A20168
:102D6E00AF50AE4FAD4EAC4D121FDD8F508E4F8D0E
:102D7E004E8C4D200A127E187F5A1227DC7E647FFD
:102D8E007CE4FBAD25122997E54E454D6016200AD1
:102D9E00107E187F5D1227DC7D03AF4EAE4D1228DC
:062DAE00BD7F00227F0141
:012DB40022FC
:0100200022BD
:10353D00300004C2000547300D04C20D054BE508EF
:10354D00B40106E4F50812365830190CE547D3944A
:0C355D00144008C219D21B22E4F54722DA
:0B364D00301B05C21B7F01227F002202
:102DC100020881E493A3F8E493A34003F68001F29F
:102DD10008DFF48029E493A3F85407240CC8C33313
:102DE100C4540F4420C8834004F456800146F6DFE2
:102DF100E4800B01020408102040809035CEE47E6F
:102E0100019360BCA3FF543F30E509541FFEE493D6
:102E1100A360010ECF54C025E060A840B8E493A39D
:102E2100FAE493A3F8E493A3C8C582C8CAC583CAC8
:102E3100F0A3C8C582C8CAC583CADFE9DEE780BE80
:0135E90000E1
:101A6B00BB010689828A83E0225002E722BBFE0279
:091A7B00E32289828A83E49322AC
:101A8400BB010CE58229F582E5833AF583E0225017
:101A940006E92582F8E622BBFE06E92582F8E22261
:0D1AA400E58229F582E5833AF583E493227B
:101AB10075F008758200EF2FFFEE33FECD33CDCCEC
:101AC10033CCC58233C5829BED9AEC99E58298406F
:101AD1000CF582EE9BFEED9AFDEC99FC0FD5F0D64C
:101AE100E4CEFBE4CDFAE4CCF9A88222B800C1B976
:101AF1000059BA002DEC8BF084CFCECDFCE5F0CBB4
:101B0100F97818EF2FFFEE33FEED33FDEC33FCEBEC
:101B110033FB10D703994004EB99FB0FD8E5E4F9A7
:101B2100FA227818EF2FFFEE33FEED33FDEC33FC94
:101B3100C933C910D7059BE99A4007EC9BFCE99A88
:101B4100F90FD8E0E4C9FAE4CCFB2275F010EF2FCD
:101B5100FFEE33FEED33FDCC33CCC833C810D707CD
:101B61009BEC9AE899400AED9BFDEC9AFCE899F808
:0E1B71000FD5F0DAE4CDFBE4CCFAE4C8F9229B
:0E1B7F00C3E49FFFE49EFEE49DFDE49CFC2277
:101B8D00EB9FF5F0EA9E42F0E99D42F0E89C45F0AE
:011B9D002225
:0C1B9E00ECF0A3EDF0A3EEF0A3EFF022BA
:101BAA00A8828583F0D083D082121BC1121BC11276
:101BBA001BC1121BC1E473E493A3C583C5F0C5839B
:101BCA00C8C582C8F0A3C583C5F0C583C8C582C885
:011BDA0022E8
:1013E800E539242DF8E6053922782A301602782DB9
:1013F800E475F001121C3C021A6B200FEB7F2ED211
:101408000F8018EF540F2490D43440D4FF30130BBE
:10141800EF24BFB41A0050032461FFE53A600215B7
:101428003A053DE53D7002053C30160D782AE47515
:10143800F001121C3CEF021BDB02348A7403D21643
:101448008003E4C216F5398B2A8A2B892CE4F53AF5
:10145800F53CF53DE53A60077F2012142380F575C9
:101468003BFFC210C20FC211C212C214C215C2176A
:101478001213F1FF700D3016057F00121434AF3DC2
:10148800AE3C22B4255FC2D5C2131213F1FF24D09B
:10149800B40A00501A75F00A783A30D50508B6FF34
:1014A8000106C6A426F620D5047002D21280D924DB
:1014B800CFB41A00EF5004C2E5D213021634D2108A
:1014C80080C6D20F80C0D21180BCD2D580BAD214C7
:1014D80080B47F201214232011077401B53A00400C
:1014E800F11213E8FF12142302145CD217D21580EC
:1014F800951213E8FB1213E8FA1213E8F94A4B7035
:101508000679057A177BFF20112EE53A602A7E00BE
:101518008E82758300121A8460060EEE653B70F0A9
:10152800C2D5EBC0E0EAC0E0E9C0E0EE12167BD01D
:10153800E0F9D0E0FAD0E0FB121A6BFF60AAEBC02A
:10154800E0EAC0E0E9C0E0121423D0E02401F9D0B9
:10155800E03400FAD0E0FBE53B0460DCD53BD98001
:10156800877BFF7A167977D211809C79108002796F
:1015780008C215C2178008D2D5790A8004790AC230
:10158800D5E53B047002F53BE4FAFDFEFF1213E8D3
:10159800FC7B082010131213E8FD7B10300F0A1291
:1015A80013E8FE1213E8FF7B20EC3382D592D55066
:1015B80013C3E4300F069FFFE49EFEE42010039D52
:1015C800FDE49CFCE4CBF8C210EC700CCFCECDCC83
:1015D800E824F8F870F38017C3EF33FFEE33FEED1D
:1015E80033FDEC33FCEB33FB994002FB0FD8E9EBFE
:1015F800301005F8D0E0C448B210C0E00AEC4D4EF7
:101608004F78207B0070C2EAB53B0040BCC0E012B6
:10161800167DD0F0D0E0201004C4C0E0C4B210C0E1
:10162800F012140CD0F0D5F0EB02145C121C9B14D1
:10163800F95315735814CA4C14C64215774F157FC1
:0F16480044157F4914DF4315855515694615690B
:101657004515694717255014CE2D14D22E14F52B96
:1016670014D62314F320170E2A148E48000014ED05
:101677003F3F3F00790AA2D5201214301409B91050
:10168700020404B9080104A2D52015025001042060
:1016970011689211B53A005034C0E07F203012191A
:1016A7007F30A21172157214500F1216D4C211C2D4
:1016B70015C214C2177F30800F301403E9C0E0123F
:1016C7001423301403D0E0F9D0E0B53ACC30141726
:1016D7007F30B9100C1214237F583013077F78809E
:1016E70003B908031214233011057F2D0214237F39
:1016F700202017F87F2B2015F322921180CF286E18
:10170700756C6C2900D2101213E83010F8C21078EB
:101717003A30D50108F602148E2D5043495812135A
:10172700E82403B405004001E49017209312141431
:0D173700743A121414D212753A040215739C
:102081008B2A8A2B892CE4F536F535F534F533F5B1
:1020910031F532E52E452F452D6012EBC0E0EAC047
:1020A100E0E9C0E0AB2DAA2EA92F121C4CAB2A05EA
:1020B1002CE52CAA2B7002052B14F9121A6BF5379B
:1020C100C394094007E537D3940D40E1E537642017
:1020D10060DBE537B42D054332038016E537B42BB9
:1020E10005433201800C74FF252CF52C74FF352B30
:1020F100F52BE53060046410703FAB2AAA2BA92CA4
:10210100121A6B64306009E530702E75300A80292F
:10211100900001121A84FF64786004EFB4581343ED
:1021210032017530107402252CF52CE4352BF52B7A
:102131008007E5307003753008AB2A052CE52CAA21
:102141002B7002052B14F9121A6BF537C3946140F9
:102151000AE537D3947A50035337DF74D02537F526
:1021610037C3940A400CE5379411406D74F9253753
:10217100F537E537D39530506043320185363B85DD
:10218100353A853439853338AF307E00E4FCFDAB18
:1021910036AA35A934A833121BEDC8ECC8C9EDC95C
:1021A100CAEECACBEFCBE4FCFDFEEB2537F536EEEC
:1021B1003AF535ED39F534EC38F533AF36AE35ADAA
:1021C10034FCAB3BAA3AA939A838D3121B8D500372
:1021D10002213A43320402213AE53220E003E4804D
:1021E1002DE52E452F452D601EAB2AE52C24FFF948
:1021F100E52B34FFFAEBC0E0EAC0E0E9C0E0AB2D2B
:10220100AA2EA92F121C4CE53230E20774FFFFFE03
:10221100FDFC22E532AF36AE35AD34AC3330E103EF
:04222100021B7F22FB
:101BDB00BB010689828A83F0225002F722BBFE01E9
:021BEB00F322E3
:101BED00E88FF0A4CC8BF0A42CFCE98EF0A42CFC97
:101BFD008AF0EDA42CFCEA8EF0A4CDA8F08BF0A415
:101C0D002DCC3825F0FDE98FF0A42CCD35F0FCEB73
:101C1D008EF0A4FEA9F0EB8FF0A4CFC5F02ECD3938
:0F1C2D00FEE43CFCEAA42DCE35F0FDE43CFC22A5
:101C3C00FAE6FB0808E6F925F0F618E6CA3AF622A9
:101C4C00BB011A89828A83D0F0D0E0F8D0E0F9D0B9
:101C5C00E0FAD0E0FBE8C0E0C0F0021CCA5016E984
:101C6C00F8D083D082D0E0F9D0E0FAD0E0FBC0828B
:101C7C00C083021CC1BBFE16E9F8D083D082D0E031
:0F1C8C00F9D0E0FAD0E0FBC082C083021CD32263
:101C9B00D083D082F8E4937012740193700DA3A3D8
:101CAB0093F8740193F5828883E4737402936860EC
:061CBB00EFA3A3A380DFEC
:091CC100EBF608EAF608E9F62248
:091CCA00EBF0A3EAF0A3E9F0221B
:091CD300EBF208EAF208E9F22242
:00000001FF
